:03800000028011EA
:20800B00438CDC05083275810890F004E4F0438901D2AFD2A9D28C128408021954058179E2
:20802B00027A0089828A83E0548078FE128673F6700302805EE61286A57BFF12869C1287B9
:20804B007645F0700302805B74FF75F0FF02806302802A740175F0001581221280287900ED
:20806B007A00740189828A83F0221280287BFF7CFF12877645F0700302808E74FF75F0FF8F
:20808B000280C779007A00743889828A83F012802879007A00740C89828A83F01280667444
:2080AB000075F000C0E0C0F0740075F000C0E0C0F01280C815811581158115812212802849
:2080CB0078FB128673E61286A590812A0286AE79007A0078F9128673E6248089828A83F082
:2080EB0002813E79007A0078F9128673E624C089828A83F002813E79007A0078F912867343
:20810B00E6249489828A83F002813E79007A0078F9128673E624D489828A83F002813E16C1
:20812B0081030002810200EE800100DA80000000003E81220581740078FE128673F678FE9A
:20814B00128673E618181818860108860275F00012869589828A83E01286A57B0012869C36
:20816B0012877F45F070030281AF800B78FE128673E604F61480C712802879017A00C0014C
:20818B00C00278FC128673E618181818860108860275F00012869589828A83E0D083D08207
:2081AB00F002817778FA128673E60886F015812212802879017A0078FB128673E689828A8A
:2081CB0083F0227F0812867F78F3128673E60886F07B007C0012875645F070030281FD7405
:2081EB000075F00079F7128678128695742DF702820D740075F00079F7128678128695743F
:20820B002BF778F3128673E60886F078FD128673F608A6F078F3128673E60886F07B007C72
:20822B000012875645F0700302825B78FD128673E60886F012874F78F3128673F608A6F0E7
:20824B0018E60886F012873C18F608A6F0128745740175F00079F712867812869578F31234
:20826B008673E60886F07BE87C031286DE2430C5F03400C5F0F718E60886F07BE87C0312E5
:20828B0086D778FD128673F608A6F0740275F00079F712867812869578FD128673E60886E6
:2082AB00F07B647C001286DE2430C5F03400C5F0F778F3128673E60886F07B647C0012863C
:2082CB00D778FD128673F608A6F0740375F00079F712867812869578FD128673E60886F03B
:2082EB007B0A7C001286DE2430C5F03400C5F0F7740475F00079F712867812869578FD1202
:20830B008673E60886F07B0A7C001286D72430C5F03400C5F0F7740075F00079F712867843
:20832B00128695E71286A5C0E0C0F01281BB15811581740175F00079F7128678128695E7A9
:20834B001286A5C0E0C0F01281BB15811581740275F00079F7128678128695E71286A5C09F
:20836B00E0C0F01281BB15811581740375F00079F7128678128695E71286A5C0E0C0F012D9
:20838B0081BB15811581740475F00079F7128678128695E71286A5C0E0C0F01281BB158188
:0783AB0015817FF802868EA8
:07800300C0D0C0E00283B20F
:2083B200C0F0C083C082C000C001C002C003C004C005C006C0071283E6D007D006D005D08D
:2083D20004D003D002D001D000D082D083D0F0D0E0D0D03290F0001287CA89828A83E090EF
:2083F200F002F090F002E01286A5C0E0C0F01281BB1581158122740075F00390F000F0A30F
:20841200C5F0F0C5F074FF90F002F0740090F003F07481F5A8E5884401F58812807574D117
:2084320075F087C0E0C0F012813F15811581740075F000C0E0C0F0740175F000C0E0C0F09D
:208452001280C8158115811581158179007A0289828A83E0542060030284B5E5B0540870F8
:208472000302847902846D74DD75F087C0E0C0F090F003E01286A5C0E0C0F0740275F0009D
:208492001284B9158115811581158190F0001287CA90F003E00490F003F01489828A83F04A
:2084B20002845D02845D2223F42581F81287A71285051287A70284D478FB12867386820809
:2084D2008683E0602D1284E3A380F778FB128673E63099FDC299F599B40A17740D80F2E4C2
:2084F20030980C3098FDC298E599B40D02740A75F0002212864C868208868308E4FEFFE06B
:20851200700612864CE4F022B42551A3E0B42D05430780A3E0B4300343074024D0B40A00F6
:20853200500BCE75F00AA42EFEA3E080EEE0B46413E60886F030F70843072012874CA6F04D
:2085520018F68003B4750543070A8021B478054307108019B46F10430708801112864CF047
:20857200A312864CA38095B462624307027A00C004C005C006C007AB0753031F7C00E608C5
:2085920086F0128706A6F018F6EDD007D006D005D0042430B43A0040022407C0E00AE64549
:2085B200F070CC12864CA902EF30E505742DF0A30A128655D0E0F0A3D9FA0808EF30E7A1ED
:2085D200EAC39E509C7420F0A30A80F4B4630DAA0112864C128655E6F0A380DEB47331C01E
:2085F20082C08386820886837A00E06004A30A80F9868318868212864C12865512864CE0E9
:20861200A312864C6004F0A380F2D005D00480AAB4691B86017A00E76004090A80F91286DD
:208632004C1286558601E76091F009A380F8F97A0112864C128655E9809ECDC583CDCCC5BD
:2086520082CC22EE601A8FF020F715C002EAC39E500C742030F6027430F0A30A80EFD002DE
:2086720022C82581C822C92581C97A0022D083D082CF2581F581CFC082C08322CF2581F52A
:2086920081CF2229F9E5F03AFA227C00CB30E7011CCB2275F00030E70215F022FDE493A3E5
:2086B200FEE493A3FF4E7009E493FE740193FF800BE493A3B5050BE493B5F0068F838E82A0
:2086D200E473A380D81287068EF0ED22C0F0C0E0E5F06C5480FF8CF030F707EB12874CAC80
:2086F200F0FBD0E0D0F030F70312874CBF80051287068046C002C001AAF0F97E007D007FC5
:2087120011C3E933F9EA33FADF08F5F0E9D001D00222ED33FDEE33FEC3ED9BF5F0EE9C4097
:20873200E0ADF0FED380DB12873C04700205F02212874514B4FF0215F022128745F4C5F0C7
:20875200F4C5F0221287894029801E12878940227017801E12878940107017800C128789C3
:208772005010800512879D6009E4F5F02212879D60F7E4F5F00422C39BC5F09C20E707201F
:20879200D207C345F02220D2F9D322C5F0C39C7003E5F09B2290F004E0A360F8E0FFA3E01A
:2087B200A3CF2582F582EF3583F58380EBFBE0CB22FCE0FBA3E0CC22FAE0F9A3E0CA2255E6
:0F87D20053422054657374696E67000A25640072
:00000001FF
